:10000000758107758920758841758DFD75985090AB
:1000100006671202E31202D91202BB784074107B09
:10002000047600081470FA1204C6540F2440F876BF
:10003000551204C6540F2440F8E6B400F476571263
:1000400004C6540F2440F8E6B400F476501204C6F7
:10005000540F2440F8E6B400F476421204C6540F5C
:100060002440F8E6B400E6764212008E1201F61241
:1000700000B0120373B402031204981203D660E9AD
:100080009007D71202D91202E31202BB808D7910B9
:100090007840E954037005740A1202B3747C1202AA
:1000A000B3E61202B30819E970E8740A1202B32227
:1000B0001202D91202D99005051202E31202D912D6
:1000C00002BBB461071202F278FF8024B464071205
:1000D000030978FF801AB4770712032278FF801093
:1000E000B4730712035178FF8006B466031200F759
:1000F0001202D9B8FFC922EB70111202D9900798E9
:100100001202E31202D9740178FF221B1203AC9091
:1001100005C11202E31202BBB4640BE95403940359
:10012000603012015622B46109E9540360241201BF
:100130007522B4730EE9C313C313C394036013127F
:10014000019422B4770CE9C313C313C360041201F2
:10015000B4221201E522E9042440F8E6C394576072
:100160000CE6C394436006E6C3945170041201D4B4
:10017000221201E522E9142440F8E6C39457600CEA
:10018000E6C394436006E6C3945170041201D4227E
:100190001201E522E924042440F8E6C39457600CD8
:1001A000E6C394436006E6C3945170041201D4225E
:1001B0001201E522E994042440F8E6C39457600C48
:1001C000E6C394436006E6C3945170041201D4223E
:1001D0001201E5229006011202D91202E31202D99D
:1001E00078FF7405229005F51202D91202E312027B
:1001F000D978FF74012278407900C3E694556004F1
:10020000090880F6E9540360031202449403600372
:10021000120250E9C313C313C3600312025C9403B8
:10022000600312026912022922FF9007C51202E33D
:10023000EB24301202B39007CF1202E31202D9125C
:1002400002D9EF22FFE92440F818E6120276EF22E5
:10025000FFE92440F808E6120276EF22FFE9244085
:100260009404F8E6120276EF22FFE924402404F811
:10027000E6120276EF22603AE6B457061202C41282
:1002800002D9B450061202CB1202D9B442061202AD
:10029000D21202D9B4510C1202C41202D91202CBEA
:1002A0001202D9B4430C1202C41202D91202D212A1
:1002B00002D922C299F5993099FD220E3098FCC2DC
:1002C00098E599229004E11202E3229004F41202CC
:1002D000E3229004D31202E322F5F0740A1202B36F
:1002E000E5F022E493600AC299F5993099FDA38064
:1002F000F2221203ACE95403700374012218E67071
:100300004176550876007401221203ACE954039437
:1003100003700374012208E670287655187600747D
:1003200001221203ACE9C313C313C3700374012287
:10033000E89404F8E6700B7655E82404F876007427
:100340000122B44203740322B450037402227404E1
:10035000221203ACE9C313C313C3940370037401E3
:1003600022E82404F8E670DA7655E89404F876007A
:10037000740122B4010674001204AF22B4020C907E
:1003800005411202E31202D9740122B4030C900554
:100390006E1202E31202D9740222B4040C90059B7F
:1003A0001202E31202D9740122740122790078400A
:1003B000C3E694556004090880F62279007840C3AA
:1003C000E694576010C3E69451600AC3E694436014
:1003D00004090880EA22600122FF1204C6540304C3
:1003E000C313C313C3B400281203BB1204C65407BB
:1003F000C313C3B400051204148015B4010512041C
:1004000041800DB4020512046F800512045D800066
:1004100060D6EF22E9607E14607B1460781460750A
:10042000142440F8E6B4000476578057B4550E9073
:1004300006241202D91202E37F0174012204F6801D
:1004400042E9941004604E04604B04604804604527
:1004500024102440F8E6B400D376578026E95403EC
:100460006033E9142440F8E6B400C176578014E9FB
:1004700054039403601FE9042440F8E6B400AD7609
:10048000578000E92440F8E6B4570576007401224D
:1004900014F67401227400221203ACE92440F876A9
:1004A000001204C6540F2440F8E670F5765522FF7A
:1004B000EB9409600F1204C65407B40507900801B5
:1004C0001202E30BEF22EEB400010475F0DDA42468
:1004D00035FE22596F752068656172206261747300
:1004E00000596F7520736D656C6C20612077756D98
:1004F00070757300596F75206665656C20612064A6
:100500007261667400506C6561736520707265730A
:100510007320772C612C732C6F72206420666F72AD
:10052000206120646972656374696F6E206F722048
:100530007072657373206620746F20666972652E11
:1005400000596F752066656C6C20696E746F206150
:10055000207069742E2020486176652061206E69C4
:1005600063652061667465726C6966652E00546807
:1005700065206261747320686176652063617272C0
:1005800069656420796F7520746F20612072616ED7
:10059000646F6D2073706163652100436F6E6772D5
:1005A0006174756C6174696F6E73212020596F7569
:1005B0002772652077756D70757320666F6F642183
:1005C00000506C656173652075736520772C612C14
:1005D000732C6F72206420746F2063686F6F736573
:1005E000206120646972656374696F6E206F662094
:1005F0006669726500596F75206D69737365642152
:1006000000596F75206B696C6C6564207468652097
:1006100077756D7075732E2E2E6E69636520776FFA
:10062000726B21005468652077756D707573206654
:100630006F756E6420796F7521212020486F706579
:1006400020796F752772652066756C6C206F662047
:10065000766974616D696E7320616E64206D696E78
:100660006572616C73210057656C636F6D652074F2
:100670006F2048756E74207468652057756D7075AD
:10068000732C20776865726520796F752068756EA8
:100690007420746865206D6F73742064616E676583
:1006A000726F7573206F660A616E7920616E696D75
:1006B000616C20746861742068617320657665726E
:1006C0002077616C6B656420746865206561727465
:1006D00068212020596F7572206F6E6C79206672C8
:1006E00069656E6420697320796F75722074727504
:1006F0007374790A626F7720616E64206172726F21
:10070000772E2020496E20746865206361766573BA
:10071000206172652070697473207468617420644C
:10072000726F7020796F7520746F20796F757220E9
:10073000646561746820616E6420626174730A7418
:10074000686174207069636B20796F752075702003
:10075000616E64206D6F766520796F7520746F20EF
:1007600072616E646F6D20706C616365732E202002
:10077000476F6F642048756E74696E67210A507206
:100780006573732061206B657920746F20636F6ED1
:1007900074696E7565210A00596F75206861766508
:1007A000206E6F206172726F77732E2E2E626574C9
:1007B0007465722074727920746F2066696E64208B
:1007C0006F6E652100596F75206861766520002085
:1007D0006172726F777300506C656173652070721F
:1007E0006573732061206B657920746F20706C6174
:1007F0007920616E6F746865722067616D65210A8A
:10080000000A0A596F7520666F756E6420616E204C
:090810006172726F77210A0A007F
:00000001FF
